:10000000382822082304031913288230831681001C
:100010008330831281000108031D0B28A203220AEA
:100020000319A30301280800121492103D3083160F
:10003000920083122208A4002308A500A41C971292
:10004000A4189716241C1712241817160310A50CB1
:10005000A40C0310A50CA40C24089500831686118B
:10006000053083129200303097050F309706080054
:1000700007309F0000308500003086008316003076
:100080008500003086000313051485146430831244
:10009000A000A101A2002108A300142005185D28DA
:1000A0001E30A0070318A10A2008A2002108A300FF
:1000B0001420FA30A200A301012085186C281E30FC
:1000C000A002031CA1032008A2002108A300142001
:0C00D000FA30A200A301012000004E281D
:02400E00183F59
:00000001FF
